:100000000C942A000C9445000C9445000C94450077
:100010000C9445000C9445000C94FA020C94450095
:100020000C9445000C94A7020C9445000C944500D8
:100030000C9445000C9445000C9445000C9445002C
:100040000C9445000C9445000C9445000C9445001C
:100050000C94450011241FBECFE5D4E0DEBFCDBF18
:1000600011E0A0E6B0E0E4E6F8E002C005900D92F1
:10007000A435B107D9F711E0A4E5B1E001C01D92A4
:10008000A736B107E1F70C94CA030C9400008091E5
:10009000660121E030E0A90102C0440F551F8A9596
:1000A000E2F780916601992787FD9095820F931F53
:1000B000B90102C0660F771F8A95E2F7CB01842B46
:1000C00080935F01109260011092610110926201B1
:1000D00080916501A90102C0440F551F8A95E2F77E
:1000E00080916501992787FD9095820F931FB90133
:1000F00002C0660F771F8A95E2F7CB01842B8093AD
:10010000630180916401E82FFF27E15AFE4F80913F
:10011000580102C0220F331F8A95E2F78081822B9B
:100120008083089582E08093640123E02093580146
:1001300091E090935901109256018093660180934B
:1001400065011092550190935A0110925701209326
:100150005E0180E49CE99BBD8ABD089580E387BB76
:1001600014BA8FEC88BB8FEF85BB8ABB81BB82E062
:1001700083BF8AE08EBD80E49CE99BBD8ABD81E19E
:1001800089BF7894089580915B01813011F48FEEDE
:1001900005C080915B018F3F19F48FED88BB0895F6
:1001A0008FECFCCF1EBC80915B01813071F410920A
:1001B0005F0180E18093600180E2809361018FE7BD
:1001C00080936201109263010DC087E480935F0108
:1001D00089E480936001809361018093620181E3EF
:1001E00080936301789420E030E087EE93E0C2973B
:1001F00097FFFDCF2F5F3F4F83E128383807ACF3DF
:1002000086B3809599278F709070892B29F480E0B0
:100210008F5F8F3FE9F7F4CFF8940E9492000E941D
:10022000AE0010925B01109257010895EF92FF9279
:100230000F931F93CF93982F9870282F2170382FEA
:10024000327010E082FF05C08091660185300CF4A9
:1002500011E000E0992329F08091660118160CF452
:1002600001E0FF24222331F080916501853014F4F0
:1002700091E0F92EEE24332331F0809165011816B8
:1002800014F481E0E82E112329F0809166018F5F3C
:1002900080936601002329F080916601815080934C
:1002A0006601FF2029F0809165018F5F80936501D1
:1002B000EE2029F08091650181508093650190E0E6
:1002C00080915501882309F491E090935501809124
:1002D0005501882309F432C180915801882329F4FB
:1002E0008091560181958093560180915801863006
:1002F00029F4809156018195809356018091640183
:10030000813019F49091660102C09091650180914D
:100310006401813029F080916401833009F0E6C0E6
:1003200080915801891779F080915801282F33273F
:1003300027FD3095492F552747FD5095CA01019655
:100340002817390731F4809159018195809359011B
:100350008FC080915801282F332727FD3095CA017F
:1003600001972817390721F480915601813071F0E7
:1003700080915801992787FD90954E5F5F4F8417B4
:10038000950779F4809156018F3F59F48091590176
:1003900081958093590180915601819580935601F2
:1003A00067C0C0916401C13061F580915B018F3FEE
:1003B00061F180915B01815080935B010E94C300D9
:1003C0008091640190915901890F8093640180911B
:1003D000580190915601890F80935801C0935A019A
:1003E0001EBC789420E030E087EE93E0C29797FF40
:1003F000FDCF2F5F3F4F83E128383807ACF3F894E7
:100400002FC080915B01813019F40E94D20099C005
:1004100080915B018F5F80935B010E94C30080919C
:10042000640190915901890F809364018091580172
:1004300090915601890F8093580181E080935A0171
:100440001EBC789420E030E087EE93E0C29797FFDF
:10045000FDCF2F5F3F4F83E128383807ACF3F89486
:100460008AE08EBD0E9492000E94C3001894F1F1B0
:1004700080916401813059F4112349F08091560133
:1004800018162CF0809156018F5F80935601809151
:100490006401813061F4002351F0809156018F3F57
:1004A00031F02CF08091560181508093560180915B
:1004B0006401833059F4FF2049F0809156011816E9
:1004C0002CF0809156018F5F8093560180916401DA
:1004D000833061F4EE2051F0809156018F3F31F06E
:1004E0002CF08091560181508093560180915801E3
:1004F000882349F4809156018F3F29F48091560159
:1005000081958093560180915801863049F48091FD
:100510005601813029F480915601819580935601CE
:100520008091640190915901890F809364018091B9
:10053000580190915601890F8093580181E0809372
:100540005A01CF911F910F91FF90EF9008951F9244
:100550000F920FB60F9211242F933F934F935F93F7
:100560006F937F938F939F93AF93BF93EF93FF937B
:10057000809154018F5F80935401809154018530A4
:1005800010F0109254011BBA2091540181E090E0C8
:1005900002C0880F991F2A95E2F7809582BB80914F
:1005A0005401E82FFF27E15AFE4F80818BBB8091D9
:1005B0005C0190915D01892B61F080915401843040
:1005C00041F480915A01882321F00E944700109243
:1005D0005A01FF91EF91BF91AF919F918F917F91C0
:1005E0006F915F914F913F912F910F900FBE0F90A0
:1005F0001F9018951F920F920FB60F9211242F93F0
:100600003F934F935F936F937F938F939F93AF939A
:10061000BF93EF93FF9380915C0190915D01892BD3
:10062000A9F1809157018F5F809357018091570105
:100630008A3041F51092570180915E018F5F80935F
:100640005E0180915E01282F332727FD3095432FCF
:10065000532F60E47CE980E090E00E94F503DA012A
:10066000C901880F991FAA1FBB1F820F931FA41FC8
:10067000B51F9BBD8ABD80915E0185361CF084E666
:1006800080935E0186B380950E941601FF91EF91E1
:10069000BF91AF919F918F917F916F915F914F919A
:1006A0003F912F910F900FBE0F901F9018951092B1
:1006B0005B010E9492000E94AE00FFCF0F931F9338
:1006C000CF93DF9310E0012FC0E0D0E080916B006A
:1006D00080935F0180916C008093600180916D0038
:1006E0008093610180916E008093620180916F0020
:1006F000809363010E94AE0086B38095282F332734
:1007000020FF21C00023E9F42197D7FF02C0C0E0F9
:10071000D0E0FE01EE0FFF1FEE0FFF1FEC0FFD1FDD
:10072000E559FF4F808180935F0181818093600153
:1007300082818093610183818093620184818093AF
:10074000630101E001C000E021FF22C01123F1F4A8
:100750002196CE32D10514F0CDE2D0E0FE01EE0FAD
:10076000FF1FEE0FFF1FEC0FFD1FE559FF4F8081AC
:1007700080935F0181818093600182818093610118
:1007800083818093620184818093630111E0B4CFFF
:1007900010E0B2CFCFE5D4E0DEBFCDBF10925F0155
:1007A0001092600110926101109262011092630137
:1007B00010925D0110925C010E94AE0086B380959C
:1007C000C82FDD27C0FF08C081E090E090935D0155
:1007D00080935C010E945703C1FFF0CF10925D012E
:1007E00010925C010E945E03E9CF97FB092E05265B
:1007F0000ED057FD04D014D00AD0001C38F4509508
:100800004095309521953F4F4F4F5F4F0895F6F734
:1008100090958095709561957F4F8F4F9F4F08956C
:10082000A1E21A2EAA1BBB1BFD010DC0AA1FBB1FF4
:10083000EE1FFF1FA217B307E407F50720F0A21B66
:10084000B30BE40BF50B661F771F881F991F1A94D3
:1008500069F760957095809590959B01AC01BD01FD
:04086000CF01089527
:1008640047494949310010207F000A3F4848483F22
:100874007F494949363E414141227F4141221C7F03
:10088400494949417F484848403E4149492E7F08EB
:1008940008087F00417F4100060101017E7F0814A2
:1008A40022417F010101017F2010207F7F10080475
:1008B4007F3E4141413E7F484848303E4145423DAC
:1008C4007F484C4A31314949494640407F40407E47
:1008D4000101017E7C0201027C7F0204027F631419
:1008E40008146360100F106043454951613E454947
:1008F400513E0010207F0047494949314249596916
:10090400460818287F0871494949463E494949061D
:1009140040474850603649494936304949493E7F45
:100924004141417F000000007F4F494949794949CD
:1009340049497F780808087F794949494F7F4949DF
:10094400494F404040407F7F4949497F794949495F
:040954007F2E0000F2
:00000001FF
